:020000040000FA
:10000000850186018316073085008601831207303B
:100010009F002E2882076F340334763457341B3404
:100020005D347D3407347F345F343F3479346C344D
:1000300073347C343C346D343934013463343834B3
:1000400068343534313471343E341F34303419342B
:1000500078346B346134653468341034A301A501FD
:10006000A4016C20051C412805193228051C4128D3
:10007000051D3628A30A213023020318A3016C2092
:100080003228A4176C20851843282130A500712040
:100090000C302307A2005620A20B4B28A4012230CB
:1000A000A50071208517612085132E28FA30A00045
:1000B000C830A10000000000A10B5A28A00B58284E
:1000C0000800FA30A000C830A10000000000A10B19
:1000D0006528A00B6328080023080A202404860052
:0C00E000080025080A20240486000800FF
:02400E00103F61
:00000001FF
